:400000007d006830303030307d01da7e7e3030307e3030307d01df7e7d01e07e7d01dd7e7e3030307e3030307e3030307e3030307e3030307e3030307e3030307e303030f9
:400040007e3030307e3030307d01de7e7e3030307d01e17e7d01e27e7e3030307e3030307e3030307e30303043320055f80055f90050034e7c01a7900862e2007c01ee8fde
:40008000ff50005502033c0203a0053f028ff8500157505502003c0202a00b08283f02187509008ff27f3030303030303030303030303030303030303030303030303030c8
:4000c0003030303030303030303030303030303030303030303030303030303030303030303030303030303030303030303030303030303030303030303030303030303000
:4001000030303030303030303030303030303030303030303030303030303030303030303030303030303030303030303030303030303030303030303030303030303030bf
:4001400030303030303030303030303030303030000070ef623200623000620500620600620700620800620900620a01620b00620c00620d00620e00620f00621000621170
:4001800000621200621300621400621500621600623d00622b00623180622a00627300711062e31370ef7f7c01ab7f7c015270ef7f105700404040404040404040404040df
:4001c000404040404040403900791900dfe7207f7840407d01d678bff97f90077e7e7e7e7e7e7e76007f4300207f4100df7f104f380243e00271018028550000500c087c88
:4002000001b138ff3c0003d02b3c0100a0095601005600008007560101560000520153013c0100b0059fc380039fbb507d087c01b138ff8fc538fe208fff30303030303069
:40024000303030303030303030303030303030303030303030303030303030303030303030303030303030303030303030303030303030303030303030303030303030307e
:40028000303030303030303030303030303030303030303030303030303030303030303030303030303030303030303030303030303030303030303030303030303030303e
:4002c00030303030303030303030303030303030303030303030303030303030303030303030303030303030303030303030303030303030303030303030303030303030fe
:4003000030303030303030303030303030303030303030303030303030303030303030303030303030303030303030303030303030303030303030303030303030303030bd
:020000040010ea
:020000040020da
:02000000291cb9
:00000001ff
